:1000000000308A0004280000840183131F30830518
:10001000193083169900A63098009030831298000A
:1000200083161F149F141F159F1107309C00FF306B
:100030008312A00083161F109F141F159F151F13F6
:1000400083121F179F1383169F1383121F1494127A
:10005000A01220088316870083122016200883161A
:1000600087008312A01120088316870001308312B5
:1000700094000030831694000108C73908388100C5
:10008000831290010030F800920000308316920035
:1000900007309C00050864000230F700F70B4E287B
:1000A00051281C0883120D1383169D014030F8005F
:1000B00083121F08C73978049F0064000630F700D8
:1000C000F70B60281F151F1963281E08A100A1083F
:1000D000031973282108313C031C7328831605116A
:1000E00083120515FA282108323C0318A428210898
:1000F0004F3C031CA42883160511831205156400C8
:100100002030F700F70B822885288316051183120B
:10011000051164002030F700F70B8C288F28831618
:1001200085118312851164002030F700F70B9628A3
:100130009928831685118312851564002030F700F5
:10014000F70BA028A328FA282108503C0318C1283F
:100150002108773C031CC128831685118312851161
:1001600064002030F700F70BB328B62883168511FA
:100170008312851564002030F700F70BBD28C028D6
:10018000FA282108783C0318F22821089F3C031C18
:10019000F228831685128312851664002030F7003A
:1001A000F70BD028D328831685128312851264009A
:1001B0002030F700F70BDA28DD288316851183122B
:1001C000851164002030F700F70BE428E728831638
:1001D00085118312851564002030F700F70BEE2897
:1001E000F128FA282108A03C0318FA288316851262
:0801F0008312851662286300EA
:02400E0039393E
:00000001FF
